:020000020000FC
:100000000C949A2018951895189518951895189588
:100010001895189518951895189518951895189578
:100020001895189518951895189518951895189568
:100030001895189518951895189518951895189558
:100040001895189518951895189518951895189548
:100050000C944E061895189518951895189518959E
:10006000189518950C94DC091895189518951895FD
:100070001895189518951895189518951895189518
:100080001895189518951895189518951895189508
:1000900018951895189518951895189518951895F8
:1000A00018951895189518951895189518951895E8
:1000B00018951895189518951895189518951895D8
:1000C00018951895189518951895189518951895C8
:1000D00018951895189518951895189518951895B8
:1000E00018951895189518951895189518951895A8
:1000F0001895189518951895189518951895189598
:100100001895189518951895189518951895189587
:100110001895189518951895189518950C943D06EE
:100120001895189518951895189518951895189567
:10013000189518950C94B20518951895189518955A
:100140001895189518951895189518951895189547
:100150001895189518951895189518951895189537
:100160001895189518951895189518951895189527
:100170001895189518951895189518951895189517
:100180001895189518951895189518951895189507
:1001900018951895189518951895189518951895F7
:1001A00018951895189518951895189518951895E7
:1001B00018951895189518951895189518951895D7
:1001C00018951895189518951895189518951895C7
:1001D00018951895189518951895189518951895B7
:1001E00018951895189518951895189518951895A7
:1001F000189518951895189518951895AA594EBEE2
:1002000034D514BEAE16863CF81D473E59298B3EA8
:10021000F81D473EAE16863C34D514BEAA594EBED4
:10022000D4D26FBCBB3CF2BC872453BD1A6DA4BDB5
:10023000AE76E6BD17740FBEB5875B3F17740FBE71
:10024000AE76E6BD1A6DA4BD872453BDBB3CF2BC9F
:10025000D4D26FBC14BEA1BD6FEDFCBDDC252FBE9A
:10026000E9383F3FDC252FBE6FEDFCBD14BEA1BDBC
:1002700001010204082A2A2A2A2A2A2A2A2A0001F3
:1002800056275527452A27021D271196260B5B2640
:1002900001AF26012A27012827011D2702AF2605C5
:1002A0004826018926019626036426029626039293
:1002B00026FB1BEC1093520018E010935000E1E570
:1002C000F0E0108113FFFBCF005400935500E0E5F0
:1002D000F0E0008100610083E1E5F0E0008104FFCF
:1002E000FBCF08ED04BF04E000934000E0E5F0E040
:1002F00000810E7F0083089501E00093280200E34F
:1003000000932902089501E00093300208E300936E
:10031000310208950DE00093200300E400932103CF
:1003200000E00093220300E40093240300EE009316
:10033000280300EE00932A0300EE00932A03089599
:100340000150104098018901232BD1F708958A9319
:10035000802F03C008EE1DEFF3DF8A95082F802F52
:100360000023C1F7899108950E94102480E090E055
:10037000A0E0B0E048E0442E1BC0442D50E0440F04
:10038000551F440F551FFA01E658FE4D008011809D
:1003900022803380442D50E0440F551F440F551FD9
:1003A000FA01E258FE4D00821182228233824A9481
:1003B00041E0441610F7EEE7F1E200831183228357
:1003C0003383442423C0042D10E0000F111F000FBD
:1003D000111FF801E450FE4F4591559165917491BC
:1003E000042D10E0000F111F000F111FF801E2583B
:1003F000FE4D00811181228133810E949522AC0142
:10040000BD010E943422C801D901439409E040167D
:10041000D0F28C019D01E5E00C9421240E9410246F
:1004200080E090E0A0E0B0E048E0442E1BC0442D06
:1004300050E0440F551F440F551FFA01E256FE4D80
:100440000080118022803380442D50E0440F551FDE
:10045000440F551FFA01EE55FE4D00821182228293
:1004600033824A9441E0441610F7E2EAF1E2008355
:10047000118322833383442423C0042D10E0000F12
:10048000111F000F111FF801E450FE4F45915591C7
:1004900065917491042D10E0000F111F000F111FC2
:1004A000F801EE55FE4D00811181228133810E94B9
:1004B0009522AC01BD010E943422C801D9014394A8
:1004C00009E04016D0F28C019D01E5E00C94212456
:1004D0000E94102480E090E0A0E0B0E04CE0442EC8
:1004E0001BC0442D50E0440F551F440F551FFA0107
:1004F000EE53FE4D0080118022803380442D50E069
:10050000440F551F440F551FFA01EA53FE4D008258
:100510001182228233824A9441E0441610F7E6ECBD
:10052000F1E20083118322833383442423C0042D0A
:1005300010E0000F111F000F111FF801E05EFD4FCA
:100540004591559165917491042D10E0000F111F94
:10055000000F111FF801EA53FE4D00811181228125
:1005600033810E949522AC01BD010E943422C80152
:10057000D90143940DE04016D0F28C019D01E5E0D5
:100580000C9421240E94102480E090E0A0E0B0E0D0
:100590004CE0442E1BC0442D50E0440F551F440F27
:1005A000551FFA01EA50FE4D0080118022803380F1
:1005B000442D50E0440F551F440F551FFA01E650DB
:1005C000FE4D00821182228233824A9441E0441619
:1005D00010F7EAEFF1E2008311832283338344248E
:1005E00023C0042D10E0000F111F000F111FF80190
:1005F000E05EFD4F4591559165917491042D10E099
:10060000000F111F000F111FF801E650FE4D008171
:100610001181228133810E949522AC01BD010E948B
:100620003422C801D90143940DE04016D0F28C0168
:100630009D01E5E00C9421240E94102480E090E0CC
:10064000A0E0B0E046E0442E1BC0442D50E0440F33
:10065000551F440F551FFA01E65DFD4D00801180C6
:1006600022803380442D50E0440F551F440F551F06
:10067000FA01E25DFD4D00821182228233824A94AA
:1006800041E0441610F7EEE2F2E200831183228388
:100690003383442423C0042D10E0000F111F000FEA
:1006A000111FF801EC5AFD4F4591559165917491D8
:1006B000042D10E0000F111F000F111FF801E25D63
:1006C000FD4D00811181228133810E949522AC0170
:1006D000BD010E943422C801D901439407E04016AD
:1006E000D0F28C019D01E5E00C9421240E9410249D
:1006F00080E090E0A0E0B0E046E0442E1BC0442D36
:1007000050E0440F551F440F551FFA01EA5BFD4DA1
:100710000080118022803380442D50E0440F551F0B
:10072000440F551FFA01E65BFD4D008211822282C3
:1007300033824A9441E0441610F7EAE4F2E200837F
:10074000118322833383442423C0042D10E0000F3F
:10075000111F000F111FF801EC5AFD4F45915591E3
:1007600065917491042D10E0000F111F000F111FEF
:10077000F801E65BFD4D00811181228133810E94E9
:100780009522AC01BD010E943422C801D9014394D5
:1007900007E04016D0F28C019D01E5E00C94212485
:1007A0000E940C2408011901842E583049F40DECE4
:1007B000402E0CEC502E0CEC602E0DE3702E15C06C
:1007C000593049F40DEC402E0CEC502E0CE4602E08
:1007D0000DE3702E0AC05A3041F40FE8402E02ECAF
:1007E000502E05EF602E0CE3702E82019301A001C4
:1007F000B1010E949522C801D901A201B30100E014
:1008000010E020E83FE30E947822482D50E0440F9A
:10081000551F440F551FFA01EA59FD4D4081518182
:10082000628173810E949522AC01BD010E94342235
:10083000482D50E0440F551F440F551FFA01EA5947
:10084000FD4D00831183228333830E94E2210E94A5
:10085000D521E9E00C941D240E940D24842FA52F9E
:100860000E94D521482F50E0440F551F440F551FBB
:10087000FA01E657FD4D40815181628173810E94EA
:100880007822280139010A2F10E020E030E00E9490
:10089000E021A801B901820193010E940E23482F93
:1008A00050E0440F551F440F551FFA01E657FD4D08
:1008B00040815181628173810E94342290E0880FCF
:1008C000991F880F991FFC01E657FD4D0083118386
:1008D00022833383E8E00C941E2420E020938004DC
:1008E00027E3F801258328E0F801218321E0F801BE
:1008F000248308950E941124D801922F832F08E5A4
:10090000FD01068304EF11E01BDDFD01978304EF79
:1009100011E016DDFD01878304EF11E011DD07E032
:1009200000938304E4E00C9422248A930C54104036
:1009300020E030E00E94E0214DEC5CEC6CE47DE3D3
:100940000E940E230E94E221802F00EA14E0C5DFFE
:1009500030E820E000EA14E0CDDF0CE211E0F0DC4A
:1009600031E320E000EA14E0C5DF39EB22E000EAE1
:1009700014E0C0DF3BE420E100EA14E0BBDF382FE5
:1009800021E000EA14E0B6DF08EB1BE0D9DC899136
:1009900008951091480001E0009348002091A000C4
:1009A0003091A2000091A2000C7F04600093A2008D
:1009B0004FB77894E8E4F0E0008101600083509143
:1009C000CD01EF93FF930F932F93EBECF1E008ED44
:1009D00021E004BF20832F910F91FF91EF9103E05D
:1009E0000093CD018895109348002093A000309388
:1009F000A2005093CD014FBF0895EFECF1E00081CC
:100A000007FDFBCF0895F9DFEFECF1E0008101FF76
:100A100011C006E30093CA01EF93FF930F932F9346
:100A2000EBECF1E008ED21E004BF20832F910F9162
:100A3000FF91EF9108959A938A93C801DEDFFC013C
:100A4000E05CF140B89750F44091362450E009E062
:100A500010E00E94E820800F911F17C0803901E04C
:100A6000900798F44091352450E000E210E00E9495
:100A7000E82098014091362450E000E610E00E9402
:100A8000E820200F311F820F931F082F0093C00111
:100A9000892F8F718093C10100E00093C20106E0AD
:100AA0000093CA01EF93FF930F932F93EBECF1E0C8
:100AB00008ED21E004BF20832F910F91FF91EF916A
:100AC0000091C4018991999108950E941224C8014E
:100AD000A22F00E00093060900E000934608FC0105
:100AE000E05CF140B89750F44091362450E009E0C2
:100AF00010E00E94E820800F911F17C0803901E0AC
:100B0000900798F44091352450E000E210E00E94F4
:100B1000E82098014091362450E000E610E00E9461
:100B2000E820200F311F820F931F6DDF03E3009336
:100B3000CA01082F0093C001892F8F718093C101D2
:100B400000E00093C201A093C40105E30093CA0131
:100B500020DF03E00093060901E000934608E3E08C
:100B60000C9423249A938A93FA93EA930A927A93A1
:100B70006A935A934A933A932A931A930A930FB615
:100B800000911524002329F4E0E0F2E000810460E4
:100B900000830091FE23039507700093FE230091CC
:100BA000FE2310E0000F111FF801EB50FD4D0081F6
:100BB000118100933A0310933B030091FE2310E050
:100BC000000F111FF801EB51FD4D008111810093C1
:100BD000380310933903009100240023B1F10091F0
:100BE000852310918623212F220F220B322F409133
:100BF000FE2350E0440F551F440F551FFA01EB5BD5
:100C0000FC4D4081518162817381400F511F621FF1
:100C1000731F4083518362837383809198239091E3
:100C200099230196809398239093992300919A2376
:100C300010919B238017910741F400E0009300245A
:100C400010E000939823109399230091152401300C
:100C500029F4E0E0F2E00081046000830FBE099116
:100C600019912991399149915991699179910990F5
:100C7000E991F9918991999118952A931A930A9378
:100C80002FB7009110021091110200938523109349
:100C900086232FBF09911991299118955A924A924A
:100CA000BA93AA939A938A93FA93EA933A922A92DE
:100CB0001A920A927A936A935A934A933A932A938E
:100CC0001A930A935FB600910024002309F05BC3D6
:100CD000009102240023B1F580E0883008F0A6C01E
:100CE00058E0482F082F10E0000F111F000F111FB0
:100CF000F801EB5BFC4D0081118122813381ACDD79
:100D00000E94E221482F50E0440F551F440F551F09
:100D1000FA01EB59FC4D008311832283338300E0F9
:100D200010E020E030E0482F50E0440F551F440F02
:100D3000551FFA01EB5BFC4D008311832283338343
:100D40008395CBCF009106240830C8F180E088302D
:100D500008F06CC050910624482F082F10E0000FB7
:100D6000111F000F111FF801EB5BFC4D0081118179
:100D7000228133810E94D52113DD0E94E221482F78
:100D800050E0440F551F440F551FFA01EB59FC4D1D
:100D9000008311832283338300E010E020E030E001
:100DA000482F50E0440F551F440F551FFA01EB5BCD
:100DB000FC4D00831183228333838395C8CF80E069
:100DC00033C0509106245395482F082F10E0000F90
:100DD000111F000F111FF801EB5BFC4D0081118109
:100DE0002281338139DD0E94E221482F50E0440FF7
:100DF000551F440F551FFA01EB59FC4D0083118319
:100E00002283338300E010E020E030E0482F50E000
:100E1000440F551F440F551FFA01EB5BFC4D008337
:100E20001183228333838395883058F20FEF009328
:100E300000248091FA239091FB2301968093FA235A
:100E40009093FB238E3100E0900719F400E00093AB
:100E500038248091F8239091F92301968093F82308
:100E60009093F923803707E1900749F400E010E000
:100E70000093F8231093F92301E0009319240091C3
:100E8000F8230F77013019F401E00093202400E0EB
:100E900010E020E030E0E8EAF3E2008311832283EF
:100EA0003383E4EAF3E2008311832283338300E097
:100EB00010E020E030E0E1E3F4E2008311832283DC
:100EC000338344249BC0042D10E0000F111F000F3A
:100ED000111FF801EB59FC4D0081118122813381F2
:100EE0000E94D521C801D901042D10E0000F111F67
:100EF000000F111FF801EB59FC4D00811181228177
:100F000033810E94D521AC01BD010E949522E1E30D
:100F1000F4E240815181628173810E943422E1E3D5
:100F2000F4E20083118322833383E4EAF3E2008155
:100F30001181228133810E94D521C801D901042D5C
:100F400010E0000F111F000F111FF801EB59FC4DAD
:100F500000811181228133810E94D521442D50E0EE
:100F6000440F551F440F551FFA01EB5FFC4D4081A4
:100F70005181628173810E949522AC01BD010E9462
:100F800034220E94E221E4EAF3E200831183228307
:100F90003383E8EAF3E200811181228133810E94E8
:100FA000D521C801D901042D10E0000F111F000F39
:100FB000111FF801EB59FC4D008111812281338111
:100FC0000E94D521442D50E0440F551F440F551F5A
:100FD000FA01EB5DFC4D40815181628173810E9479
:100FE0009522AC01BD010E9434220E94E221E8EA70
:100FF000F3E20083118322833383439408E0401695
:1010000008F461CF40E050E060E071E4E1E3F4E235
:1010100000811181228133810E940E230E942E2A99
:10102000E1E3F4E2008311832283338300919E2362
:1010300010919F2320E030E00E94E021A801B90137
:10104000E1E3F4E200811181228133810E940E23C9
:101050000E94E22100939623109397230091FC2392
:1010600010E0F801E059FD4F449150E000919623C3
:10107000109197230E94FC200093962310939723AE
:10108000E4EAF3E20081118122813381E4EBF3E2AF
:101090000083118322833383E8EAF3E20081118124
:1010A00022813381E8EBF3E20083118322833383CF
:1010B000E0ECF3E20081118122813381E4EBF3E281
:1010C0004081518162817381041715072607370714
:1010D0007CF4E0ECF3E200811181228133810F5F27
:1010E0001F4F2F4F3F4F00831183228333830EC046
:1010F000E0ECF3E200811181228133810150104044
:10110000204030400083118322833383ECEBF3E2F1
:101110000081118122813381E8EBF3E2408151812A
:101120006281738104171507260737077CF4ECEBFF
:10113000F3E200811181228133810F5F1F4F2F4F16
:101140003F4F00831183228333830EC0ECEBF3E225
:1011500000811181228133810150104020403040B4
:1011600000831183228333830091FF230023D9F06E
:1011700000E00093FF23E4EBF3E200811181228180
:101180003381E0ECF3E20083118322833383E8EBC5
:10119000F3E20081118122813381ECEBF3E20083E1
:1011A000118322833383E0ECF3E2008111812281F9
:1011B0003381E4EBF3E24081518162817381401B12
:1011C000510B620B730B4083518362837383ECEB8F
:1011D000F3E20081118122813381E8EBF3E2408167
:1011E000518162817381401B510B620B730B4083F1
:1011F000518362837383E4EBF3E2008111812281E6
:101200003381E4EEF3E20083118322833383E8EB3E
:10121000F3E20081118122813381E8EEF3E2008361
:1012200011832283338300910224013009F07BC0B3
:1012300000911124013029F5E4EBF3E200811181E2
:10124000228133810E94D5210E94B4010E94E221B3
:10125000ECEDF3E20083118322833383E8EBF3E2C6
:1012600000811181228133810E94D5210E940E02CA
:101270000E94E221E0EEF3E20083118322833383B4
:101280006AC000911124023029F5E4EBF3E20081F9
:101290001181228133810E94D5210E9468020E941F
:1012A000E221ECEDF3E20083118322833383E8EB48
:1012B000F3E200811181228133810E94D5210E94B5
:1012C000C2020E94E221E0EEF3E200831183228356
:1012D000338341C0009111240330E9F5E4EBF3E2DC
:1012E00000811181228133810E94D5210E941C033B
:1012F0000E94E221ECEDF3E2008311832283338329
:10130000E8EBF3E200811181228133810E94D52133
:101310000E9476030E94E221E0EEF3E20083118353
:101320002283338318C0E4EBF3E200811181228130
:101330003381ECEDF3E20083118322833383E8EB06
:10134000F3E20081118122813381E0EEF3E2008338
:10135000118322833383ECEDF3E20081118122813A
:101360003381ECEAF3E20083118322833383E0EEDE
:10137000F3E20081118122813381E0EBF3E200830B
:1013800011832283338301E000930D245FBE099112
:1013900019912991399149915991699179910990BE
:1013A000199029903990E991F99189919991A99190
:1013B000B9914990599018954A92BA93AA939A93E1
:1013C0008A93FA93EA933A922A921A920A927A9319
:1013D0006A935A934A933A932A931A930A934FB66D
:1013E00000E010E000932524109326248091A008AB
:1013F000813489F4E8E3F4E200810160008300E0D5
:1014000010E00093FA231093FB23E4E6F6E000815A
:1014100002600083B1C500913824002309F4ACC5F3
:1014200000913824033031F400913824002309F06E
:1014300021C4A2C58434F9F401E2CBD500918923FB
:10144000D0D500919123CDD5ECEAF3E20081118152
:1014500045E00E94F620C5D5E0EBF3E20081118162
:1014600045E00E94F620BDD500911E24BAD500E0CB
:1014700000933824D9CF833571F4009109240A955B
:1014800000930924002319F401E00093092400E0EB
:1014900000933824C9CF843571F400910924039551
:1014A00000930924053118F004E10093092400E0B9
:1014B00000933824B9CF863471F400911124039538
:1014C00000931124043018F001E00093112400E08F
:1014D00000933824A9CF873509F05EC00E947E169C
:1014E00001E277D50E94E8127CD54FE050E00091F0
:1014F0009623109197230E94FC2073D5009111240C
:1015000070D5009109246DD5009110246AD5009101
:10151000922367D50091362464D50091352461D596
:1015200000911A245ED5E0918723F09188233196AB
:10153000AF01652F660F660B762F00E81DE82BE5DF
:1015400030E00E94732100932B2410932C240091EF
:101550002B2410912C241A930A9324E231E20EECEE
:1015600012E20E94132A22960EEC12E21AD5009182
:10157000942337D50091932334D50091962310916D
:101580009723083E23E0120718F401E00093FF239D
:1015900000E00093382448CF853409F06DC00E94E4
:1015A0007E1601E216D5009136241BD50091352414
:1015B00018D500911A2415D50091062412D5009152
:1015C00017240FD50091FC230CD50091072409D5D1
:1015D0000091142406D50091122403D50091012412
:1015E00000D500911324FDD400910824FAD4009171
:1015F0000A24F7D400911C24F4D400911B24F1D4C4
:10160000E0918723F09188233196AF01652F660F13
:10161000660B762F00E81DE82BE530E00E94732171
:1016200000932B2410932C2400912B2410912C2414
:101630001A930A9324E231E20EEC12E20E94132A7A
:1016400022960EEC12E2ADD4EFE3F1E200811181BB
:10165000228133813A932A931A930A9329E231E241
:101660000EEC12E20E94132A24960EEC12E299D498
:1016700000E000933824D8CE8B3299F400918E2369
:10168000B0D400918F23ADD44FE050E00091962369
:10169000109197230E94FC20A4D400E000933824EA
:1016A000C3CE8F3649F4E4E8F6E000810B7F008377
:1016B00000E000933824B8CE893709F043C001E236
:1016C00088D4009136248DD4009135248AD4009199
:1016D0001A2487D4E0918723F09188233196AF01B3
:1016E000652F660F660B762F00E81DE82BE530E0CE
:1016F0000E94732100932B2410932C2400912B24FF
:1017000010912C241A930A9324E231E20EEC12E297
:101710000E94132A22960EEC12E243D40091EC238D
:101720001091ED231A930A932EE231E20EEC12E2AD
:101730000E94132A22960EEC12E233D400E00093AA
:10174000382472CE853741F5E0918723F0918823C4
:101750003196AF01652F660F660B762F00E81DE806
:101760002BE530E00E94732100932B2410932C244E
:1017700000912B2410912C241A930A9324E231E235
:101780000EEC12E20E94132A22960EEC12E209D409
:1017900000E00093382448CE893631F4D8D621D4DD
:1017A00000E00093382440CE813791F40091022468
:1017B000013021F400E00093022403C001E0009313
:1017C000022401E00093FF2300E0009338242CCE94
:1017D0008E36F1F400919523002349F401E0009343
:1017E0009523E4E4F6E000810160008308C000E096
:1017F00000939523E4E4F6E000810E7F00832091BE
:10180000952302EF11E061D900E0009338240CCE5B
:10181000823671F4009144060F7000934406E4E6AA
:10182000F6E000810D7F008300E000933824FCCDBA
:10183000803579F408E00093A4080FE00E94A70126
:1018400008E10093A4088091A00800E000933824E8
:10185000EBCD8636D9F5E7E8F3E20081118101503E
:1018600010400083118300918723109188230093F7
:10187000260910932709E0918723F0918823319658
:10188000AF01652F660F660B762F00E81DE82BE58C
:1018900030E00E94732100932B2410932C2400919C
:1018A0002B2410912C241A930A9324E231E20EEC9B
:1018B00012E20E94132A22960EEC12E272D301E089
:1018C0000093FF2300E000933824AECD8736D9F58E
:1018D000E7E8F3E2008111810F5F1F4F008311835E
:1018E00000918723109188230093260910932709DC
:1018F000E0918723F09188233196AF01652F660F21
:10190000660B762F00E81DE82BE530E00E9473217E
:1019100000932B2410932C2400912B2410912C2421
:101920001A930A9324E231E20EEC12E20E94132A87
:1019300022960EEC12E235D301E00093FF2300E083
:101940000093382471CD883659F50E947E16E8D36D
:10195000E0918723F09188233196AF01652F660FC0
:10196000660B762F00E81DE82BE530E00E9473211E
:1019700000932B2410932C2400912B2410912C24C1
:101980001A930A9324E231E20EEC12E20E94132A27
:1019900022960EEC12E205D300E00093382444CDE9
:1019A0008B3631F5E091EC23F091ED233197E09304
:1019B000EC23F093ED23FF2332F408E611E00093CB
:1019C000EC231093ED2364D60091EC231091ED23CA
:1019D0001A930A932EE231E20EEC12E20E94132ACD
:1019E00022960EEC12E2DDD200E0009338241CCDEA
:1019F0008A3641F5E091EC23F091ED233196E093A6
:101A0000EC23F093ED23E83601E0F00734F000E03A
:101A100010E00093EC231093ED233AD60091EC23D1
:101A20001091ED231A930A932EE231E20EEC12E2AA
:101A30000E94132A22960EEC12E2B3D200E0009329
:101A40003824F2CC8C36B9F40E947E16A9D30091CA
:101A5000EC231091ED231A930A9323E331E20EEC69
:101A600012E20E94132A22960EEC12E29AD200E0B1
:101A700000933824D9CC873759F40E947E16009100
:101A80001A24023009F4B8D200E000933824CCCCF8
:101A9000843641F507E00093062401E00093172403
:101AA00006E00093132401E00093FC2302E000937E
:101AB000072402E00093122401E00093142401E0C3
:101AC0000093012401E00093082402E1009309241B
:101AD00008E000930A2408E500931C2400E000932A
:101AE0003824A2CC813339F401E000930E2400E0C5
:101AF0000093382499CC823311F500E010E0009374
:101B0000F6231093F7230093F4231093F52320E09A
:101B100000E110E00E94650520E001E110E00E9474
:101B200065052091F6233091F7230091F42310915D
:101B3000F5230E94C21600E00093382475CC893347
:101B400081F500911C24039500931C240B3518F09B
:101B50000AE500931C2400911C2410E011950195C6
:101B60001040212F220F220B322F0E94D52143E358
:101B700053E365E672E40E940E230E94A32AA801A3
:101B8000B90100E010E020E83FE30E940E23EFE3FC
:101B9000F1E2008311832283338300E00093382431
:101BA00043CC883381F500911C240A9500931C24B2
:101BB000063418F406E400931C2400911C2410E061
:101BC000119501951040212F220F220B322F0E94D8
:101BD000D52143E353E365E672E40E940E230E949D
:101BE000A32AA801B90100E010E020E83FE30E9429
:101BF0000E23EFE3F1E2008311832283338300E0BD
:101C00000093382411CC873379F50E9406160BEE29
:101C100011E00E941B05B02FA0E00CEE11E00E9425
:101C20001B0510E0A02BB12BA093A223B093A323FC
:101C30000091A2231091A3231A930A9329E331E27E
:101C40000EEC12E20E94132A22960EEC12E2A9D1A7
:101C500003EF11E00E941B05C4D101E00093FF23B4
:101C600000E000933824E0CB03E000933824809315
:101C7000372482C100913724063371F400911A246D
:101C8000023009F479C1282F0DEE11E00E9465059C
:101C900000E00093382470C100913724053309F027
:101CA00045C000911A24023009F466C103EF11E027
:101CB0000E941B0510E000932B2410932C24E0912C
:101CC0002B24F0912C24369734F008ED04BF01E06A
:101CD0000093790051C1282F0EEE11E00E94650596
:101CE0000E947E1600911A247CD120912B242395EA
:101CF00003EF11E00E9465052091F8230BEF11E03E
:101D00000E9465050E94AD28202F0AEE11E00E9476
:101D1000650500911A24023029F425E504EF11E04D
:101D20000E94650500E00093382426C10091372405
:101D3000063531F48093102400E0009338241CC150
:101D4000009137240A35F1F4809392230091922375
:101D5000083531F4009124060C7F009324060EC050
:101D60000091240603600093240608EE1DEF0E94F4
:101D7000A0010091922310E00E94950400E00093DE
:101D80003824FAC000913724093481F4803150F4AA
:101D9000809313244091132450E008E710E00E9440
:101DA000E820DED200E000933824E6C0009137241A
:101DB000073459F4843028F48093FC230091FC23E9
:101DC000BBD600E000933824D7C0009137240235F9
:101DD000E1F48234B1F42FEF0AEF11E00E946505BF
:101DE0002FEF0BEF11E00E94650500E510E037D3FF
:101DF00000E61AEE0E94A00108ED04BF01E0009386
:101E0000790000E000933824B7C0009137240037F0
:101E100081F480933624209136240AEF11E00E9449
:101E2000650500E0009338249CD600E00093382438
:101E3000A3C000913724033749F5809335242091BE
:101E400035240DEF11E00E946505882331F40091DF
:101E5000640608610093640614C0813059F4E4E616
:101E6000F6E000810F7E0083E4E6F6E00081086082
:101E7000008307C0823029F400916406077E009336
:101E800064066FD600E00093382476C000913724B2
:101E9000083441F48B3010F48093062400E0009362
:101EA00038246AC000913724033641F4843010F49A
:101EB0008093172400E0009338245EC000913724FB
:101EC0000A3739F402E00093072400E00093382435
:101ED00053C0009137240D3441F4843010F48093C2
:101EE000142400E00093382447C0009137240234C2
:101EF00041F4853010F48093122400E000933824DC
:101F00003BC000913724013641F4833010F48093B4
:101F1000012400E0009338242FC0009137240437B7
:101F200061F4883010F480930824009108240E9402
:101F3000EF1700E0009338241FC0009137240837C2
:101F400041F48A3010F480930A2400E0009338248E
:101F500013C0009137240D3661F490E0880F991F6B
:101F60008093EC239093ED2393D300E000933824E7
:101F700003C000E0009338244FBE099119912991C4
:101F800039914991599169917991099019902990C4
:101F90003990E991F99189919991A991B9914990D3
:101FA00018950E941124C801A0E007C0B0E0FC0110
:101FB000EA0FFB1F008115D0A395B0E0FC01EA0FEA
:101FC000FB1F0081002311F0AD3080F3E4E00C949E
:101FD0002224E1EAF8E0108115FFFBCF0093A0086E
:101FE0000895013209F400E4E1EAF8E0108115FFF8
:101FF000FBCF0093A008089500911A24023009F045
:102000008EC030918823232F01E010E00E946505E7
:102010002091872302E010E00E9465053091ED23B6
:10202000232F05E010E00E9465052091EC2306E0D7
:1020300010E00E946505209106240DE110E00E9449
:102040006505209117240BE110E00E9465052091A1
:1020500013240CE010E00E9465052091FC2304E1AC
:1020600010E00E946505209107240EE110E00E9417
:1020700065052091142403E110E00E94650520917C
:10208000122407EF11E00E946505209101240FE161
:1020900010E00E9465052091102406EF11E00E94D7
:1020A00065052091922308EF11E00E9465052091BB
:1020B000082409E010E00E9465052091092403E04E
:1020C00010E00E94650520910A240CE110E00E94B6
:1020D0006505209111240DE010E00E946505209116
:1020E0001C2408E010E00E9465053091F523232FA1
:1020F0000EE010E00E9465052091F4230FE010E04F
:102100000E9465053091F723232F00E110E00E9423
:1021100065052091F62301E110E00E946505089510
:102120000E941124A0E0B0E000E0009300088BE2E0
:1021300091E012C0809326099093270900E61AEED9
:102140000E94A00104D2A017B10728F4D8018093FF
:1021500087239093882305968D3E02E0900750F3E5
:102160000091872310918823009326091093270953
:1021700066D400911A24023081F430918823232FF1
:1021800001E010E00E9465052091872302E010E045
:102190000E94650501E00093FF23E4E00C942224F3
:1021A0000E940D2400E0009300080091A0230E94EB
:1021B000A70180E090E0A0E01DC0E0EBF3E2008129
:1021C0001181228133810E94D521A801B9012A0100
:1021D0003B01ECEAF3E200811181228133810E940C
:1021E000D521A201B30172D1800F911F04E10E9499
:1021F000A701A395A53008F345E050E08C010E94AB
:102200001421C801E091EC23F091ED23E81BF90BB8
:10221000E65AFF4FE093EC23F093ED230091EC237B
:102220001091ED23093621E0120744F0ECEEF3E2C1
:102230000081118108561140008311831091ED2314
:10224000112342F4ECEEF3E20081118108591E4F94
:102250000083118300911A24023069F43091ED2338
:10226000232F05E010E00E9465052091EC2306E095
:1022700010E00E9465050CD201E00093FF23E8E026
:102280000C941E240E941124D80180E090E02AC002
:102290000DE210E0AC010E94E820F801EA0FFB1FFC
:1022A000E83601E0F00714F0E856F1408F01212FE5
:1022B000220F220B322F0E94D52145E35AEF6EE800
:1022C0007CE30E9495220E946029AC01440F551FB7
:1022D000440F551FFA01EB5FFC4D008311832283ED
:1022E00033830196883000E0900794F2E4E00C9488
:1022F00022240E941124D80180E090E02AC00DE23F
:1023000010E0AC010E94E820F801EA0FFB1FE8365C
:1023100001E0F00714F0E856F1408F01212F220F61
:10232000220B322F0E94D52145E35AEF6EE87CE361
:102330000E9495220E949620AC01440F551F440F25
:10234000551FFA01EB5DFC4D00831183228333831B
:102350000196883000E0900794F2E4E00C94222487
:102360000E940D24D80180E090E034C08D01212F1F
:10237000220F220B322F0E94D521280139018C0116
:10238000212F220F220B322F0E94D5214BED5FE02F
:1023900069E47FE30E9495220E946029A201B301B3
:1023A0000E949522280139018D01212F220F220B35
:1023B000322F0E94D521A201B3010E9434220E9433
:1023C000E2219C01220F331FF901EB50FD4D0083E8
:1023D00011830196883000E0900744F2E8E00C9405
:1023E0001E24B8014091102450E089010E94E82089
:1023F0000D3B22E0120714F00CEB12E023E22093D5
:10240000010824E02093000800932A0810932B0869
:10241000609326087093270808950E941124D8011C
:1024200004E00093000888E090E012C0409110247E
:1024300050E08C010E94E82000932A0810932B089A
:10244000A0932608B093270803E00E94A7010197F4
:10245000813000E0900754F7E4E00C9422249801C6
:1024600003E2009301084091102450E00AE010E0DC
:102470000E94E82000932A0810932B0804E610E03D
:10248000A9010E94E820009326081093270804E081
:102490000093000844E650E00091872310918823C0
:1024A0000E9414210E5F0E94A70100E00093000823
:1024B00008958A93812F10E0D2DF00E315E70E9490
:1024C000A001082F10E0CBDF899108950E942E20F3
:1024D00040E050E064E672E40E9495220E94E2210E
:1024E00008950E940D24C801D9012A013B01A201CF
:1024F000B3012A013B010091FD2310E020E030E010
:102500000E94E021A801B901820193010E940E23DB
:10251000AC01BD010E943422A201B3010E942E2011
:1025200040E050E064E672E40E9495220E94E221BD
:102530000B3520E0120714F00AE510E0063A2FEF01
:10254000120714F406EA1FEFE8E00C941E240E9420
:10255000112480E090E000E00093220200E000936C
:10256000010205E00E94A701A0E0B0E019C00CE361
:1025700010E00E94A001E0E0F2E00081086000832A
:1025800000912B020023E1F301E000932B02009164
:10259000120210911302801791070CF4C8011196D2
:1025A000A43F01E0B0071CF300E10093010202E048
:1025B00000932202835D9040992312F480E090E022
:1025C00042E050E08C010E941421E4E00C942224AB
:1025D000E0E0F2E00081006100830091330200231B
:1025E000E1F301E00093330240910C2450E00091AC
:1025F0001402109115020E94FC202091152430E055
:10260000220F331F220F331F020F131F08950E9442
:1026100011240EE210E0DDD2802F0FE210E0D9D2BB
:10262000482F502F8A01212F220F220B322F0E9478
:10263000D52140E04093010241E040930202E0E0F6
:10264000F2E040814062408340913B024423E1F349
:1026500041E040933B02A801B90100E010E02EEAFE
:1026600033E40E940E23C801D90100911602109193
:10267000170220E030E00E94E021AC01BD010E9481
:1026800095220E94E2210C521140E4E00C94222495
:102690000091EC231091ED23F5DD0091EC231091D6
:1026A000ED2327DE08950091EC231091ED23EADD60
:1026B0000091EC231091ED231CDE4091132450E097
:1026C00008E710E00E94E8204BDE0091872310917C
:1026D0008823009326091093270908959A938A93D3
:1026E00001E010E00E941B05902F80E002E010E066
:1026F0000E941B0510E0802B912B809387239093E1
:10270000882305E010E00E941B05902F80E006E082
:1027100010E00E941B0510E0802B912B8093EC238E
:102720009093ED230EE010E00E941B05902F80E0B7
:102730000FE010E00E941B0510E0802B912B80938E
:10274000F4239093F52300E110E00E941B05902FE5
:1027500080E001E110E00E941B0510E0802B912B2E
:102760008093F6239093F72303E010E00E941B056B
:10277000009309240CE110E00E941B0500930A2439
:1027800004E110E00E941B050093FC2303E110E02C
:102790000E941B050093142409EF11E00E941B0501
:1027A00000930B2407EF11E00E941B0500931224F5
:1027B0000CE010E00E941B05009313240CEF11E0C5
:1027C0000E941B0500930C2402EF11E00E941B05E0
:1027D0000093952306EF11E00E941B05009310243F
:1027E0000DE010E00E941B05009311240AE010E0A8
:1027F0000E941B05802F90E00BE010E00E941B055B
:10280000102F00E0802B912B809321249093222481
:1028100009E010E00E941B050093082400910824A1
:10282000093040F400E010910824112319F00060F1
:10283000002341F001E00093082421E009E010E0CA
:102840000E9465050EE110E00E941B05009307241D
:102850000EEF11E00E941B05009305240DE110E02E
:102860000E941B05009306240BE110E00E941B054B
:102870000093172408EF11E00E941B050093922398
:102880000FE110E00E941B050093012408E010E016
:102890000E941B0500931C2405EF11E00E941B05FC
:1028A00000931B24E1E2F4E200810160008389913E
:1028B000999108950E941124C801A9E000910A2469
:1028C000A01B06E51091892311230AF485C02091ED
:1028D0008923322F330F330B10E0201731070CF010
:1028E0007BC04AE0009189230E94D820402F4A5F94
:1028F00000912124109122240E94F62001700023CF
:1029000009F06AC000911224013029F49C010CE105
:1029100015E267DD91C0009112240230B9F40091F4
:10292000892305312CF49C0100E21EE45ADD84C0A9
:10293000009189230B342CF09C010CEA1DE051DD41
:102940007BC09C0100E717E14CDD76C000911224AA
:102950000330B9F49C01C901ABE0B0E000918923D8
:10296000102F110F110B4AE050E00E941421A01B00
:10297000B10B04E115E0AD010E94E8209C0131DDBE
:102980005BC000911224043081F49C010EE610E03B
:1029900040918923542F550F550B041B150B42E80A
:1029A00050E00E94E8201DDD47C09C01C901009154
:1029B0008923102F110F110B4AE050E00E941421BF
:1029C000F801E552FD4D418150E006E910E00E941A
:1029D000E8209C0106DD30C000918923002362F5C8
:1029E000B0E00091F0231091F123A017B10724F576
:1029F000A4E04CEE009189230E94D820A01B4A2F0E
:102A000000912124109122240E94F62001700023BD
:102A100099F443E050E08C010E94FC20C801009131
:102A200089230D3E2CF09C0100E21EE4DADC04C098
:102A30009C0100EE1BEAD5DCE4E00C9422240E9409
:102A4000112480918723909188230196AC01652FF2
:102A5000660F660B762F00E01CE62CED32E00E943C
:102A6000732148E050E060E070E00E947321C801EB
:102A7000D90148EE53E060E070E08C019D010E94B6
:102A8000732108500093182481380EE3900700E06A
:102A9000A00700E0B00724F001E00093152403C074
:102AA00000E00093152408E010E020E030E0AC01E5
:102AB000BD010E94282140E750E060E070E00E94E4
:102AC000732100939C2310939D2345E000919C2348
:102AD00010919D230E94F02040E250E00E94E820E7
:102AE00000939C2310939D2343E250E000919C238C
:102AF00010919D230E94FC2000939E2310939F23FE
:102B000000919C2310919D2300939A2310939B2363
:102B100046E150E00091152410E0401B510B00915C
:102B20008723109188230E9414210093A0231093DF
:102B3000A123E4E00C94222410912002137E109330
:102B400020020A95000F000F10912002102B109305
:102B5000200200E61AEE0E94A00101E00093FF238C
:102B60000895BCDD6CDF2091F6233091F7230091AE
:102B7000F4231091F52306D196DD0091FC23DCDFD0
:102B8000009108242CD200911C2410E0119501958D
:102B90001040212F220F220B322F0E94D52143E318
:102BA00053E365E672E40E940E230E94A32AA80163
:102BB000B90100E010E020E83FE30E940E23EFE3BC
:102BC000F1E2008311832283338301E00093FF232A
:102BD000089522E02093CA01F801049000E00093D8
:102BE000CA01002D08959A938A9390E088E005C069
:102BF000082F10E0EEDF900F83958631C8F39923FC
:102C000009F493E0092F8991999108950E94122463
:102C10000BEE11E00E941B050F3F09F04EC00CEEB9
:102C200011E00E941B050F3F09F047C0DCDFA02F19
:102C3000EEDC8091F82320918523820F209196234A
:102C4000820F800F90E003C00E94AD2893959817E3
:102C5000D8F30E94AD28802F853008F489E5282F0D
:102C60000BEE11E00E9465052A2F0CEE11E00E9488
:102C7000650520E00DEE11E00E94650520E00EEEF6
:102C800011E00E94650520E003EF11E00E94650558
:102C90000E94AD28202F0AEE11E00E9465050E94D7
:102CA000AD28202F09EE11E00E9465050E94AD2895
:102CB000202F00EF11E00E946505E3E00C9423242F
:102CC0009C01A801CA01892F90E04F7F50708C01B0
:102CD0000E94E820080F191FC801840F951F07964E
:102CE000982F80E00FEF10E0041B150BA8014F7F19
:102CF0005070842B952B8C01C90108950E941124DA
:102D00000BEE11E00E941B05B02FA0E00CEE11E0CD
:102D10000E941B0510E0A02BB12B0DEE11E00E94CC
:102D20001B05902F80E00EEE11E00E941B0510E0C5
:102D3000802B912B8D01C4DF08171907A9F453DFED
:102D4000202F30E00FEF10E08F7F9070081B190BE1
:102D50002017310749F401E000931A2400911A2446
:102D6000039500931A240BC001E000931A240091EC
:102D70001A240A9500931A2401E000931A24E4E02F
:102D80000C9422240E940B244801D90180E090E099
:102D900046C00DE210E0AC010E94E820A801480DF9
:102DA000591D483601E0500714F0485651408D0136
:102DB000212F220F220B322F0E94D5212801390109
:102DC0008A01212F220F220B322F0E94D5210801C8
:102DD000190145E35AEF6EE87CE3800191010E94FE
:102DE00095220E946029A201B3010E949522280128
:102DF00039018D01212F220F220B322F0E94D52164
:102E0000A201B3010E9434220E94E2219C01220F00
:102E1000331FF901EB51FD4D00831183019688307A
:102E200000E090070CF4B5CFEAE00C941C249A93D0
:102E30008A9300E081DE20E030E000E010E0A2DFD5
:102E4000009143211091442100933B2410933C2492
:102E50000CE00E94A701009196231091972304365D
:102E600020E0120708F4A3C088EE9DEF00E010E018
:102E700000933D2410933E2408C0EDE3F4E200816A
:102E800011810E5F1F4F0083118300913D2410912B
:102E90003E24083621E0120734F520914321309179
:102EA000442100913D2410913E246CDF03E00E94F8
:102EB000A701009196231091972308171907E8F6A8
:102EC000809196239091972300913D2410913E2468
:102ED0000093392410933A24E0919623F09197239C
:102EE000B89758F641C088EE9DEF0AE010E0B7DAD7
:102EF00000E010E0009343211093442108C0E3E474
:102F0000F1E200811181065F1F4F00831183009160
:102F1000432110914421083E27E012072CF520910F
:102F20004321309144210091392410913A242ADF21
:102F300003E00E94A70100919623109197230817A0
:102F40001907E8F6809196239091972300914321E9
:102F50001091442100933B2410933C24E09196234C
:102F6000F09197237E9758F620913B2430913C2492
:102F70000091392410913A2405DF00913B241091EF
:102F80003C240093F6231093F723009139241091E9
:102F90003A240093F4231093F5230091FC23CCDD15
:102FA00000E513EC0E94A00102E310E058DA8991D9
:102FB0009991089500EB0093010202E2009302024E
:102FC00003E00093040203E00093200208E2009370
:102FD0002102E0E0F2E00081016000830895013009
:102FE00051F401E010E800932124109322240AE018
:102FF0000093FD230895023051F40FE110E800938F
:1030000021241093222408E00093FD230895033027
:1030100051F40FE110E8009321241093222402E0E0
:103020000093FD230895043051F40FE510E8009358
:1030300021241093222400E10093FD2308950530FC
:1030400051F403E010EC009321241093222404E0B7
:103050000093FD230895063051F40FED10E800931E
:1030600021241093222400E10093FD2308950730CA
:1030700049F40FED18E9009321241093222400E174
:103080000093FD2308950E941124F89403E00E9408
:10309000590100912006036000932006009140062C
:1030A000006F00934006009160060863009360067D
:1030B00000914006036000934006009160060660A0
:1030C00000936006E0E8F6E000810460008308E118
:1030D0000093900604E10E94A701E4E8F6E0008175
:1030E000046000830AEF11E00E941B050F3F09F006
:1030F000E7C00BEF11E00E941B050F3F09F0E0C095
:1031000000E00093362405C0009136240395009317
:10311000362400913624043008F0C3C000E0009348
:10312000352413C0FC01EB58FD4F24918C01005451
:103130001E4F0E9465050196893000E0900790F3CC
:1031400000913524039500933524009135240330F4
:10315000D8F621E001E010E00E94650523EF02E0CF
:1031600010E00E94650520E005E010E00E94650582
:1031700024EB06E010E00E94650524E608EF11E06C
:103180000E94650520E00EE010E00E94650520E049
:103190000FE010E00E94650520E000E110E00E94D1
:1031A000650520E001E110E00E9465052FE003E0E5
:1031B00010E00E94650528E00CE110E00E94650522
:1031C00021E004E110E00E94650520E009EF11E034
:1031D0000E94650525E00CE010E00E94650521E0F5
:1031E0000DE010E00E94650522E007EF11E00E946B
:1031F000650521E00AE010E00E94650520E80BE08B
:1032000010E00E9465052FE20CEF11E00E946505B9
:1032100021E009E010E00E94650524E106EF11E0DD
:103220000E94650520E00DEF11E00E94650521E098
:103230000EEF11E00E94650521E002EF11E00E940F
:10324000650527E00DE110E00E94650521E00BE136
:1032500010E00E94650521E00EE110E00E94650586
:1032600020E005EF11E00E94650520E00AEE11E084
:103270000E94650520E20EEF11E00E94650528E539
:1032800008E010E00E94650521E003E110E00E94E3
:10329000650521E00FE110E00E94650580E090E007
:1032A0004BCF20E00AEF11E00E94650520E00BEF14
:1032B00011E00E94650525E003EF11E00E9465051D
:1032C0000AEF11E00E941B0500933624009136247A
:1032D000043040F000E00093362420E00AEF11E0D3
:1032E0000E9465050DEF11E00E941B050093352437
:1032F00000913524033040F000E00093352420E0B5
:103300000DEF11E00E9465052CDC009135240023AF
:1033100031F40091640608610093640617C00091BF
:103320003524013059F4E4E6F6E000810F7E008395
:10333000E4E6F6E000810860008308C002E0009344
:10334000352400916406077E0093640608EE1DEFA5
:103350000E94A00103E20093010800E0009300082E
:1033600001E00093000900918723109188230093C6
:1033700026091093270903E0009306090091A20093
:1033800007600093A20007E00093400804ED11E0FD
:10339000009366081093670801E0009346080E94B6
:1033A0008A0100919300043019F400E10093220394
:1033B000E1E4F6E000810860008303E00093A508E3
:1033C0000FE60093A60802EF0093A70808E1009318
:1033D000A40800E10093A308E2EAF0E000810160A4
:1033E000008300E00093372400914406006F0093AF
:1033F000440600919523002331F4E4E4F6E00081D3
:103400000E7F008305C0E4E4F6E0008101600083E4
:1034100000919223083531F4009124060C7F00932B
:1034200024060EC00091240603600093240608EED3
:103430001DEF0E94A0010091922310E00E949504CC
:10344000E4E6F6E000810460008302E30E94A70145
:10345000B1DD00E210E0BDDB00930C0201E210E000
:10346000B8DB00930D0202E0009322020E94830168
:103470000E947C0118D900ED17E00E940D1200EAAD
:103480001FE00E940D1200E41FE10E940D1202E0F5
:103490000E94A70100ED17E00E940D1200E00093CA
:1034A00000080091A023102F02E0109F002D0E9421
:1034B000A701E4E6F6E000810B7F008304EF11E052
:1034C0000E941B050535B1F11CE308E20E94591268
:1034D0000E94A71240919623509197230E94E820C2
:1034E00000932B2410932C24EBE2F4E20081118151
:1034F0000F7F10700083118300912B2410912C24D6
:10350000023420E0120761F000E020912B2430917A
:103510002C24263610E0310719F00060002329F032
:103520002FEF0AEF11E00E9465052FEF0BEF11E07E
:103530000E946505E3DB78940091FC23FDDAE4E664
:10354000F6E000810260008302E00E94A70101E032
:103550000093FF2300E0009319240AE00093042461
:103560000093032400E010E020E030E0E8EDF3E217
:103570000083118322833383ECECF3E20083118315
:103580002283338300938A2301E010E000932324F5
:103590001093242401E00093022400E000931624F9
:1035A00008EA0093902300938F2305E210E00E9425
:1035B0002F1202E00E94A70105E210E00E942F12E4
:1035C00004E10E94A7012FC000E117E20E94A001C0
:1035D0008091252490912624019680932524909310
:1035E0002624893F0AE29007F4F000E010E00093FF
:1035F00025241093262400E000930008009144063F
:103600000F7000934406E4E6F6E000810D7F00832E
:103610000091962310919723083E23E0120718F497
:1036200001E00093FF2300910D240023E1F300E06B
:1036300000930D240AE010E00E94A00100911924DB
:103640000130A9F400E000931924009193230B3377
:1036500048F00091942303950093942300E0009395
:10366000932305C00091932303950093932304E1D2
:1036700010910924011B00931D24009102240130A4
:1036800009F0EDC1ECEAF3E200811181228133817E
:10369000E4ECF3E20083118322833383E0EBF3E273
:1036A0000081118122813381E0EDF3E200831183F7
:1036B00022833383E0EDF3E20081118122813381A3
:1036C0000E94D521C801D901E4ECF3E20081118107
:1036D000228133810E94D521EFE3F1E240815181C3
:1036E000628173810E949522A801B9018C019D011C
:1036F0000E9478220E94E2210093EE231093EF2390
:1037000000910824043079F4E4ECF3E200811181A3
:103710002281338135952795179507950093F223DC
:103720001093F32306C00AE510E00093F2231093F0
:10373000F32300911D24102F110F110B2091EE2364
:103740003091EF23021713070CF048C100911D249C
:10375000102F110F110B2091F2233091F323021738
:1037600013070CF03BC100E00093032400910424F4
:10377000039500930424073018F001E00093FF2321
:10378000E8ECF3E20081118122813381E4ECF3E281
:103790004081518162817381401B510B620B730B1D
:1037A0004083518362837383E4EDF3E200811181EE
:1037B00022813381E0EDF3E24081518162817381A6
:1037C000401B510B620B730B4083518362837383E5
:1037D000E4ECF3E20081118122813381E4ECF3E235
:1037E00040815181628173810E942821C801D901E1
:1037F000E0EDF3E24081518162817381E0EDF3E21B
:1038000000811181228133810E942821800F911F24
:10381000A21FB31F8C019D010E94D5210E942E2A58
:103820000E94E22143E00E94F62000932724109397
:10383000282410912824112392F42EE130E004EF83
:103840001EE70E94F11108EB1BE00E94A00109E0B5
:10385000009391230EE110E00E945A1410C00091D1
:10386000272410912824212F220F220B322F0E946F
:10387000D5210E94FF270E94E22100939123E0EDD1
:10388000F3E200811181228133810E94D521A801B8
:10389000B901CA01DB01E4ECF3E20081118122816C
:1038A00033810E94D521AC01BD010E9471120093A9
:1038B00089230091292410912A242091EE2330910C
:1038C000EF2302171307A4F40091892300938B239D
:1038D000009127241091282400932324109324245A
:1038E0000091EE231091EF230093292410932A24B2
:1038F0000091892310918D23011724F400918923CD
:1039000000938C2300918C2300938D2300918B23B3
:1039100000938E230093892300918923075A033152
:10392000F0F400918923102F110F110B2091902397
:10393000322F330F330B021B130B44E050E00E9475
:10394000142110919023010F00938F2300918F2356
:103950000093902300918F230A9500938F238091E9
:10396000EE239091EF2302968C01212F220F220B40
:10397000322F0E94D5210E94FF270E94E22110E0F1
:103980000093F0231093F123009117241091042445
:10399000011708F001C200910124002329F40EE16F
:1039A00010E00E945A14F8C100910124013059F42A
:1039B00005E010E04091F0235091F1230E94E820AF
:1039C0000E945A14E9C10091EE231091EF2315953E
:1039D0000795159507950E945A14DEC100E00093E3
:1039E000010800E000930008E4E4F6E000810D7FA8
:1039F0000083E4ECF3E20081118122813381E8EC61
:103A0000F3E20083118322833383E0EDF3E200814C
:103A1000118122813381E4EDF3E20083118322835B
:103A2000338300E00093912310E000932924109346
:103A30002A2400E010E00093232410932424009310
:103A40008A23009389230AE500938C2300E00093E6
:103A50000424009103240395009303249DC1ECEA00
:103A6000F3E20081118122813381E4ECF3E20083EF
:103A7000118322833383E0EBF3E200811181228101
:103A80003381E0EDF3E20083118322833383E0EDA1
:103A9000F3E200811181228133810E94D521C80186
:103AA000D901E4ECF3E200811181228133810E948B
:103AB000D521EFE3F1E240815181628173810E945F
:103AC0009522A801B9018C019D010E9478220E94D3
:103AD000E2210093EE231093EF2300910824043099
:103AE00079F4E4ECF3E20081118122813381359590
:103AF0002795179507950093F2231093F32306C09B
:103B00000AE510E00093F2231093F3230091EE23D3
:103B10001091EF23212F220F220B322F0E94D5214B
:103B20000E94FF270E94E2210093F0231093F123CB
:103B300000911D240595102F110F110B2091EE23DC
:103B40003091EF23021713070CF0F5C000911D24EC
:103B5000102F110F110B2091F2233091F323021734
:103B600013070CF0E8C000E0009303240091042444
:103B7000039500930424E8ECF3E200811181228193
:103B80003381E4ECF3E24081518162817381401B17
:103B9000510B620B730B4083518362837383E4ED9B
:103BA000F3E20081118122813381E0EDF3E2408173
:103BB000518162817381401B510B620B730B4083F7
:103BC000518362837383E4ECF3E2008111812281EB
:103BD0003381E4ECF3E240815181628173810E9480
:103BE0002821C801D901E0EDF3E2408151816281D1
:103BF0007381E0EDF3E200811181228133810E9423
:103C00002821800F911FA21FB31F8C019D010E94CC
:103C1000D5210E942E2A0E94E22143E00E94F62034
:103C20000093272410932824109128241123D2F4E0
:103C300029E130E004EF1EE70E94F11100EA1FE0E5
:103C40000E94A00129E130E008E91AE34091EE2347
:103C50005091EF235595479555954795041B150BA6
:103C60000E94F11100910424083088F103E010E073
:103C70004091F0235091F1230E94E820980108E63A
:103C800012E44091EE235091EF23559547955595B9
:103C90004795041B150B0E94F111E0EDF3E2008142
:103CA0001181228133810E94D521A801B901CA0165
:103CB000DB01E4ECF3E200811181228133810E9477
:103CC000D521AC01BD010E9471120093892300919E
:103CD000292410912A242091EE233091EF230217FA
:103CE0001307A4F40091892300938B2300912724C8
:103CF0001091282400932324109324240091EE2370
:103D00001091EF230093292410932A2400918B23F0
:103D1000009389230091272410912824212F220F1A
:103D2000220B322F0E94D5210E94FF270E94E22100
:103D30000093912331C000E000930008E4ECF3E22B
:103D40000081118122813381E8ECF3E20083118349
:103D500022833383E0EDF3E20081118122813381FC
:103D6000E4EDF3E2008311832283338300E010E06B
:103D70000093292410932A2400E010E000932324C8
:103D8000109324240093912300E0009304240091D5
:103D9000032403950093032400910324003F41F082
:103DA00010E000910424003F19F010601123A9F0E5
:103DB00000E010E0009323241093242400938A232E
:103DC0000093892300E00093912310E000932724BF
:103DD0001093282401E00093FF2300918923102FE2
:103DE000110F110B00932B2410932C24809123246A
:103DF0009091242403968C01212F220F220B322F25
:103E00000E94D5210E94FF2740E050E060E87FEB50
:103E10000E9434220E94E22100932D2410932E242C
:103E2000E091EE23F091EF2337972CF000912B24B3
:103E300000938A2309C000918A23102F110F110BC0
:103E400000932B2410932C24E091EE23F091EF2388
:103E50003B970CF4ABC040912D2450912E2400913F
:103E60002B2410912C240E94142142E050E00E9447
:103E7000142100931F2480918B23982F990F990B65
:103E800000918D23102F110F110B801B910B0396A6
:103E90008C01212F220F220B322F0E94D5210E944C
:103EA000FF270E94E22100932F24109330240091D9
:103EB0001F24102F110F110B40912F2450913024EB
:103EC0000E94142100931F2400912B2410912C2474
:103ED000063520E012073CF042E000911F240E94CA
:103EE000D82000931F2400912B2410912C24809122
:103EF000182490E0C296081719079CF00091182426
:103F000010E0015C1F4F20912B2430912C240217CC
:103F100013073CF042E000911F240E94D820009338
:103F20001F2410912E2411231AF400E000931F2463
:103F300000911F2400231AF400E000931F24009135
:103F40001F240B301CF00AE000931F2400911F2453
:103F5000102F110F110B20913E21322F330F330BF5
:103F6000021B130B42E050E00E94142110913E21ED
:103F7000010F00931F2400911F2400933E21009104
:103F80001F2400933E2100912B2410912C2420917A
:103F90002D2430912E24020F131F012B19F400E061
:103FA00000931F2400911F2400931E2400912524B8
:103FB00010912624043620E0120741F4E8E8F6E0E8
:103FC000008103FD03C001E000930F24E8E8F6E060
:103FD000008103FF1CC000910F240130C1F40AE0EE
:103FE0000E94A701E8E8F6E0008103FF10C000E8A6
:103FF00010E00E942F1200E610E00E942F120AE04B
:104000000E94A701E4E8F6E000810B7F00830091A5
:104010000E24013049F400E000930E2400E310E088
:104020000E942F120E94171700912024013009F0DE
:10403000CBCA00E000932024E4E6F6E000810460AF
:10404000008300E117E20E94A001E4E6F6E00081AF
:104050000B7F0083BDCA00008895FECF0E940D240F
:10406000C801D9012A013B015CD057D071F482010B
:10407000930153D051F401E2EFE3F4E20083418372
:104080000FEF1FEF2FE73FE73DC044D0A201B30180
:104090000E943422AC01BD0140D061F442D03AD03C
:1040A0000E94AF230BED1FE029EC10F43FE32AC080
:1040B0003FEB28C0A201B3012DD00E940E230801BE
:1040C00019012FD0820193010E94972323D0A0F4DD
:1040D0001CD050F424D0A801B9010BED1FE029E455
:1040E00030E40E9478220EC01AD04BED5FE069E404
:1040F00070EC0E94342206C008D010F410D002C028
:104100000ED03058E8E00C941E240E94AF238001AA
:10411000910108958C019D0108950C948D230C94B8
:10412000C42840E050E060E070E008953F7741E04F
:104130000C94632903E20DBF01E20EBFC0E0D1E29F
:104140000E948228002311F00E9446290E944318F1
:104150000E942B200C942B200D01DA0140E050E04E
:1041600060E070E00E948D2339F400E010E04D9390
:104170004C9320E030E00CC0B901660F771F7E57EA
:10418000572F550F550B7D935C932F7730783F63F6
:10419000D00108950024E8E0EA9532F0001F001CE9
:1041A0000416D0F3041AF8CF001F402D009508958F
:1041B000FF27442312F4F1604195002312F4F09597
:1041C00001950E94CA20F0FD0195F1FD41950895E9
:1041D000149F102D059F100D049F002D110D0895A3
:1041E0004A951AF016950795FBCF08954A951AF04F
:1041F00015950795FBCF089500241124EFE0001FCB
:10420000111F001C111C0416150610F0041A150AC3
:10421000EA95AAF7001F111FA001009510950895B7
:104220005195419550400895FF27552312F4F160B0
:10423000F7DF112312F4F09507D00E94FC20F0FD67
:1042400003D0F1FDEDCF089511950195104008952B
:104250002224349F302D259F300D169F300D079F4F
:10426000300D249F202D310D159F200D311D069FEF
:10427000200D311D149F102D210D321D059F100D95
:10428000211D321D049F002D110D221D321D089588
:104290004A952AF03695279517950795F9CF0895F1
:1042A000002411241001E0E2EA9592F0001F111F92
:1042B000221F331F001C111C221C331C0416150660
:1042C0002606370688F3041A150A260A370AECCFA1
:1042D000001F111F221F331FA001B101009510956F
:1042E000209530950895FF27772312F4F16015D0BB
:1042F000332312F4F09509D00E945021F69508F46A
:1043000004D0F69508F409C00895309520951095CD
:1043100001951F4F2F4F3F4F089570956095509511
:1043200041955F4F6F4F7F4F0895FF27112477FB13
:10433000660F771F089409F4771F679517F8EE2723
:10434000002437FB220F331F089409F4331F2795ED
:1043500007F8089527FD0EC0EE0F001F111F221F42
:104360003A953230B8F7332319F427FD31E002C013
:1043700027FF30E0E03821F400FF08940EF4889421
:104380000F4F1F4F2F4F3F4F323038F4332319F464
:1043900027FD31E002C027FF30E03F3F29F0220F28
:1043A000000C379527950895ACC0032E002012F419
:1043B0000E948521E02F012F122F232F3EE9D1CF1C
:1043C0000024F8CFBCDF432F4F5748F04F3148F05F
:1043D00007FC91C03FE72FEF1FEF0FEF0895332742
:1043E0008CC0322F212F102F0E2F4F5141950E943C
:1043F000482107FE08950C948521F901EE0FFF1F57
:1044000037FBFF3F31F0EF2BE12BE02B8894B89482
:104410000895E02BE12B21F008949894B894089526
:104420009894889438940895FB01EE0FFF1F77FB52
:10443000FF3F31F0EF2BE52BE42B8894B8940895DF
:10444000E42BE52B69F3E8CFEFDF68F021F43723A5
:10445000262F8A010895372FFBCFE6DF20F00BF0DF
:1044600008957327EAF751C0C8DFE8F3B3F361F3A7
:10447000DBDFC8F383F3A1F358DF4017510762076E
:10448000730731F4011411F10024E89488942BC0CF
:1044900078F0332E372F732D322E262F632D312EA9
:1044A000152F532D302E042F432D302C012C132C7F
:1044B000371739F0669557954795F795E04073950E
:1044C000F7CFE7FBEE0FE0E010246AF0EF0F041FD8
:1044D000151F261F60F4279517950795E79508F493
:1044E000689433953ECFEF0B040B150B260B39CF99
:1044F000E0E87E27B9CF302D30782227112700271A
:1045000008953FE7302920E8F9CF3FEF2FEFF6CFAE
:104510008BDFD8F3D1F370783727089585DFA8F3C0
:10452000A3F3F9CF3078372793CF67DF70F383F3A6
:10453000A9F37ADF50F3B3F3A9F3F7DE0124E8948B
:104540003F57E040370FEF1F12F0D9F603C03A3E55
:1045500090F26894E0E00A92AA933A93AA2733244F
:1045600022243327049FF001059FF00D712D731F46
:10457000149FF00D711D221C069F700D211C331C11
:10458000159F700D211C331E249F700D211C331E9E
:10459000169F200C311CAA1F259F200C311CA31F25
:1045A000269F300CA11D39915EF43395A695379462
:1045B00027947795F795E79533953130BCF316C07E
:1045C000AA2322F0332351F4339510C0339571F4AC
:1045D000A991099096CFA7FD09C03A95EE0FFF1F4C
:1045E000771F221C331CAA1F3230A8F7E894FE2B39
:1045F00009F068942A2F8101E72FA9910990BACE7A
:1046000013DF10F00BF087CF80CF0EDFE9F3E0F37C
:10461000032E072670CF032E072673CFEEDEA0F3FE
:104620007BF399F301DF80F39BF3A9F37EDE012492
:1046300027FD06C0000F111F221F3150E040F8CFA8
:1046400067FD06C0440F551F661F7150F040F8CF3C
:10465000E894371BEF0B3158EF4F2AF0EE23E9F6C1
:104660003F3FD9F203C03A3EA8F26894E0E0F0E0A0
:104670001124139440175107620738F0315008F4A1
:104680006894000F111F221FEE1F041B150B260B31
:10469000EF0B000F111F221FEE1F0A9279E17A958E
:1046A000AAF0041715072607EF0730F0041B150BB7
:1046B000260BEF0B089401C08894111C221C331C9C
:1046C000001C000F111F221FEE1FE9CFF0F9E89424
:1046D000E22BE12BE02B09F06894069437942794A1
:1046E0001794E79508F468947395B9F30990332308
:1046F00011F0F0FF09C0369427941794E79508F459
:10470000689433953130BCF3012D122D232D32CE18
:104710008BCE98940895189408956FDED0F3C1F36A
:1047200083DEB8F3041715072607370708957CDEE4
:10473000A0F063DE90F029F0E32FE7273AF4731737
:10474000089572DE51F04EF008940895041715078D
:104750002607370719F016F4B8F78894089564DE31
:10476000E0F34BDED0F3E7DFC0F3089408957591D2
:10477000659155914591159011FA259035900895C0
:10478000F9DF041B10E003C0F4DF041B150B20E06D
:1047900030E005C0ECDF041B150B260B370BB8F01F
:1047A00010FC17C045910590E00FF11F041710058C
:1047B00040E02407340758F436F404910024F10152
:1047C000E01BF0090994E00FF11F25903590F101ED
:1047D000099411F4D6F7F1CF31960EF0319650E0EE
:1047E00060E070E045914B3F48F089F34F3F29F07E
:1047F0004E3F11F07591659155914591041B150B34
:10480000260B370B39F318F3E7CFFA92EA92DA92D4
:10481000CA92BA92AA929A928A927A926A925A9278
:104820004A92BA93AA939A938A930895FF84EE8446
:10483000DD84CC84BB84AA84998488847F806E8044
:104840005D804C80BB81AA8199818881F0E0EC0F6A
:10485000FD1FEF0108950E940524C1D37A015B0179
:104860006B018824992450D157D130F160E070E079
:104870000E948D23D1F50989002309F449C08E14C3
:104880009F044CF40CEF80160FEF900624F000E02C
:10489000088BE818F9080FEFE00EF01E0A890023D4
:1048A000A9F100E0098B34C027D10E940E2397D3D1
:1048B0000AE0800E00E0901E47EB53E46AEB71E5DE
:1048C0002AD190F325D160E271E425D1A0F60E94AF
:1048D0000E2385D301E0800E00E0901EF3CF0CD1B3
:1048E0007CD306EF800E0FEF901E40E057EE6BED8D
:1048F0007EE207D1A0F308D104D108F0BCCF60E27A
:1049000071E46BD30FEF800E901EF5CF01E00A8BA0
:104910000889002319F06624772444C09920EAF41A
:10492000DDD02701E0D06624772404C0D7D00FEF74
:10493000E00EF01E4FD3861497041CF40E2D0F29A1
:10494000A9F70FEF1FEF04191509801691060CF453
:1049500073C077246624639425C0340171946194F4
:1049600000E0700A1FC0DAD00E94E221402E212F01
:10497000220F220B322F0E94D521A801B901CED0DF
:104980000E947822A801B90100E010E020E231E4A1
:1049900024D3042D005DA3D0930101E0F6D2232B94
:1049A00009F4A1D0E614F704F4F6B2D060EA70E49A
:1049B000B2D008F041C044244394C6010197FC01E1
:1049C00000810E3251F0040D00830A3329F400E314
:1049D00000834424439401C044240197AE16BF06CB
:1049E00070F340FA4EF508890023B1F0C60102C009
:1049F00000830197A816B90658F4FC0102910E3203
:104A0000FC01B1F732970081FC0100830197F1CFDF
:104A100001E0800E941E0DC001E0C00ED41EC60140
:104A200005C0FC010291FC0100830197A816B9069C
:104A3000C0F301E3F50100830989002311F408C0E4
:104A4000C6D2F60102910033D9F30E3209F4BFD277
:104A500008890023C1F1F601019399203AF40DE28F
:104A60003FD09194819400E0900A02C00BE238D0CC
:104A7000442455240AE0C00ED41C01E06FD251D06A
:104A8000405DF60141936F014CD04801012BA9F71D
:104A900002E0401600E0500684F33201820117D094
:104AA0002081830114D0E40DF51D3B9720830FEF87
:104AB000400E501E01E0401600E050067CF706EF65
:104AC000C00E0FEFD01E8601E3E10C941624119561
:104AD00001951040F601E00FF11F089500E3F60183
:104AE00001936F0108950E2D0F2919F40A890023EF
:104AF00011F00EE2F5DF089549EF52E065E170E54F
:104B000008950CD00C94972303D060E87FE30895B8
:104B100040E050E0089502D00C94AF238C019D0139
:104B200008954AE050E084010C9414210E94052469
:104B3000EF97EF976A972A873B87488759876801DD
:104B40007B0100E00D830E8302C005D20ED229D274
:104B5000053249F00023C9F70D811E81EF96EF96CB
:104B60006A96E0E1B2CF0081053221F42BD2F3D175
:104B700005E2ECCF00E00C830B830A8309833E013E
:104B800002E103D205E411E2088B198B06C009810A
:104B9000002311F40081098315D2FBD10052B9F32F
:104BA000035059F00850B1F3025019F0035049F086
:104BB0000CC00A8103950A83EFCF0B8103950B8309
:104BC000EBCF0C8103950C83E7CF00810A3279F497
:104BD000B6D1AD90BD90AFD1BB203AF4B194A194C1
:104BE00000E0B00A0A8103950A83ECD114C0AA241C
:104BF000BB244AE050E00DC021916F0185010E9465
:104C0000E820A22EBB24A00EB11E00EDA00E0FEFD7
:104C1000B01EC2D188F30A81002311F000E00C839A
:104C2000B8D10E32F1F4CED1B4D10A3231F487D1F9
:104C30008D909D9080D1C6D117C0882499244AE0D8
:104C400050E0AAD188F421916F0184010E94E820EC
:104C5000822E9924800E911E00ED800E0FEF901E83
:104C6000F0CF88248A94982C80E093D10C5421F0C2
:104C70000C5131F0045039F481E0C80EA5D103C0C5
:104C800001E0C00ED81E8DD1EEE7F2E00C94C023F7
:104C900080FB5EF44D815E81652F660F660B53D1FC
:104CA000408351836283638352CF2D813E814BD1F8
:104CB000208331834CCF43D10D9111963CD10A8B87
:104CC0002E0103E14BD1FAC03AD16D907D9033D1E2
:104CD000062D072921F406E5602E01E2702E9920A9
:104CE00022F400E1802E07E2902E80E090E001C0E7
:104CF0000196F30101913F01002319F088159905F0
:104D0000BCF368D12301919581959040680E791E7E
:104D1000D5C00B81002331F0082D092919F49924FD
:104D20008824839405E611E2088B198B08810037EB
:104D300039F405D1F6D000E122D100E009832BC07F
:104D4000FDD01EF4F4D04BD101C0EBD008810F365A
:104D500011F408E0F1CF053771F70AE0EDCFEED09E
:104D60004D915D9126F46D917D91E5D005C0E3D024
:104D7000652F660F660B762FCA01DB0177234AF495
:104D80000DE209839095A095B09581959F4FAF4F07
:104D9000BF4F0AE0F4D03E0107E9F7D02E0107E942
:104DA000DDD0082F092B0A2B0B2B11F001E001C0DD
:104DB00000E00F83082D092919F40F8100FF17C0A7
:104DC000FAD0E889F989E00DF11D0081F301029321
:104DD0003F01F1D004D1012B022B032B89F799203D
:104DE00032F40C81002319F0FDD001C0DFD08E0118
:104DF00009561F4F91D0D4F30B81002309F45EC0F4
:104E00000F8100FF5BC00881083711F0083549F4B5
:104E1000E1D0F30108810083DDD000E3F3010083DA
:104E20004DC00F3609F04AC0F3010081003309F488
:104E300045C000E302933F0141C081E00881025078
:104E40000883082D092939F499248824839408C0FB
:104E500000E0088380E099201AF406E0802E99246F
:104E60006ED065D055DE60E070E00E94972328F494
:104E70004DE24983732F7058372F3E0142E1640E93
:104E8000751E6A0C7B1C4B814A938A934A814A9314
:104E9000B301A401E0DC28010C81002379F0A2D049
:104EA00082013AD05CF482D0FBCF91D006E7602E2D
:104EB00001E2702E09E7402E01E2502E42018618D1
:104EC0009708A814B9041CF480E090E007C090D0C3
:104ED000A818B90810E0A01AB10AC5010A81002378
:104EE00021F401C03FD00197EAF70981002339F08E
:104EF00032D004C030D0F30101913F0136D00FEF22
:104F0000800E901EBAF70A81002309F420CE019783
:104F10000AF41DCE27D0FBCF06191709081519056D
:104F200008958D919D9107D0A0E0B0E008950D9176
:104F30001D912D913D91A083B183089580FBF701D0
:104F4000A081B1810895F701A081B1810D911D91DA
:104F5000F2DFF8010895288539850895400E00E0B4
:104F6000501E08952885398500E2EA85FB8509955C
:104F70000D811E810F5F1F4F0D831E83089510E06A
:104F80000C871D871E871F870895600E00E0701E26
:104F90000895F60100810895F601008100530A305A
:104FA0000895F60101916F010883089500E3F3016C
:104FB00002933F0108954C855D856E857F85AEDD4A
:104FC0000C94502101E0C00E00E0D01E08950FEFB8
:104FD000C00EFBCF0FEF600EDACF0E949522C80102
:104FE000D901089505D010E04501801A910A08956D
:104FF0000981002311F001E0089500E008950E9466
:105000000924229741E050E060E070E00E9497237D
:1050100060F440E00E948D2321F402E26BD03FEF68
:105020005FC001E267D03FE75BC0AE010E94AC20E9
:10503000C801D90143EF54E065E37FE30E94972361
:1050400068F437FBAA0FBB1FB395B695A795B7F9C0
:1050500008811981015010400883198340E050E015
:1050600060E87FEB43D02801390140E050E060E880
:105070007FE33CD0A801B901820193010E940E2375
:10508000C801D901A801B9012FD02801390108812F
:10509000102F110F110B212F312F0E94D52148E124
:1050A00052E761E37FE320D04801590142E252E92F
:1050B00064ED7EE38201930117D04DED5BE96AE276
:1050C0007FE316D0A201B3010FD044E050E060E0CE
:1050D00070E40ED0AC01BD0107D0A401B50108D029
:1050E0002296ECE00C941A240C9495228C019D01DC
:1050F0000C943422EFE3F4E2008351830FEF1FEFAF
:105100002FE7089501E008950E941124C801D901F4
:105110001A013F7740E856E968E17BE40E94AF233B
:1051200038F416D0B38300E010E020E030E00DC08A
:105130003B2F0E94E2210E94D5210AD03383A8018F
:10514000B9018C019D010E947822E4E00C94222494
:10515000F10100831183228308954DE65EE466EC3D
:1051600071E4EAE7F1E200811181228133810E943A
:105170002821075C1F4C2F4F3F4F00831183228350
:10518000338389011F7708950E940524C801D9013E
:10519000BF7741E050E060E87FE33B2F0E94972318
:1051A00070F440E00E948D2329F40BED1FE029E408
:1051B0003FE350C0CC24DD24EE24FF241CC00BEDC3
:1051C000C02E0FE0D02E09E4E02EF72E40E07FEB5A
:1051D000082F48D02801390140E050E060E87FE323
:1051E0008C019D013FD0A801B901820193010E9469
:1051F0000E23C801D901AC01BD018C019D012DD048
:105200002801390144E25FEF6BE27CEB26D048E8ED
:1052100054E466EA7EE328D048E150EC6FE370E4A2
:1052200023D045EB1CD0480159014AEE54EB66E807
:1052300070E48201930118D046EB11D0A801B901A6
:10524000840195010E940E23AC01BD0106D0A60188
:10525000B70108D0E0E10C9416240C9495225DEF80
:1052600068E670E40C943422FDDFA201B301F5CFAF
:1052700020E006D0E9F70895259102D0E9F70895D6
:105280002D9301501040202F212B089584E596E5A1
:10529000FC0105911491FC013296A591B491FC0199
:1052A000349625913491422F432B19F0F901E4DF14
:1052B00001C0DEDF069616E58036910748F30895B3
:1052C00040E00C9463290E940D242897802FB32F6F
:1052D000442E40E050E060E070E00E94972310F41C
:1052E00001E001C000E0000F400EBF7743E859EF36
:1052F00062E27FE3082F3B2F80D076D041E05CEF65
:105300006FE777E40E94AF2388F5AE010E948428FE
:105310006BD0042D10E06BD0488159816A817B816C
:1053200072D0088319832A833B83AE014C5F5F4FA1
:105330002A0140E050E060E87EE35FD0A2010E94D5
:10534000842840E050E060E870E40C811D812E81EB
:105350003F8153D0A801B901088119812A813B817D
:105360000E9478220E94E221402E0CC00E94E2217D
:10537000602E3DD0A801B9018C019D0133D0460CAF
:1053800003E0402240FA3EF4AC01BD0100E010E031
:1053900020E83FE327D002E0401608F0B0588C0127
:1053A0009D0129D0280139014BEF57ED6EE179E3DA
:1053B00024D045E656E269E97BEB21D048E554E389
:1053C00063EA7DE31CD041EE5DE565E27FEB17D03B
:1053D0004BED5FE069EC7FE316D00DD02896E8E056
:1053E0000C941E240E947822C801D901089520E05F
:1053F00030E00C94E021AC01BD010C94952203D067
:10540000A201B301FACF0C9434221B2F6A2FF901A9
:10541000A081B181AD014F5F5F4F408351830C93F9
:10542000A62FB12F0895BA93AA9324970A831B83BA
:1054300089019E012A5F3F4F28833983BE01AE0157
:105440004E5F5F4F25E03AE20E94962520E0AA8158
:10545000BB812C932496A991B99108950E940924A7
:1054600022974801590141E050E060E070E00E945D
:10547000972398F440E00E948D2329F400E010E087
:1054800020E030E04EC001E2EFE3F4E2008351831C
:105490000FEF1FEF2FE73FE744C0AE010E94AC20A3
:1054A000C801D90145EC53E062E47FE30E94342255
:1054B0004AE151E562E17FE33BD0A801B9018C01EB
:1054C0009D013BD0402E088100FF14C00A952DD0CD
:1054D000802F43EF54E065EB7FE3042D0E9495227B
:1054E00037FB220F331F380F3695279537F9C80140
:1054F000D9010BC01AD0842D912FD90137FBAA0FE7
:10550000BB1FB00FB695A795B7F940E050E060E833
:105510007EE38C019D010CD0AC01BD01840195019D
:105520000CD02296ECE00C941A2442E00C94D82083
:105530000E9495222801390108950E940E23A2019C
:10554000B3010C9434220E940B242497B32F992486
:1055500040E050E060E070E00E949723882408F467
:105560008394BF7743E859EF62EA7FE33B2F62D031
:10557000AE010E9484286BD080FA442440F801E0F8
:10558000402653D00E94E22103700A9529F00A9523
:1055900031F00A9531F007C04FD0939404C0842CA9
:1055A000FCCF4AD0842CAC01BD018C019D0142D0BE
:1055B000088319832A833B8344E556E768E471EC4A
:1055C00039D040E759ED63E52DD0280139014DE38D
:1055D00054ED6EE872EC29D00E9434224881598142
:1055E0006A817B8127D045E15EED66E81BD0A8018A
:1055F000B901820193010E940E23AC01BD011AD0B2
:1056000026D090FA36F4A801B9011CD00E940E23CE
:105610001ED080FA0EF4B0588C019D012496EAE069
:105620000C941C2473E40C943422088119812A817F
:105630003B8108950C949522AC01BD0103D00E94DA
:10564000782205C000E010E020E83FE30895C8019B
:10565000D90108955A0024216056C3027E2100001A
:10566000253035640025303566002530336400254B
:1056700030336420002530345800010AD7A3BC2CF5
:1056800001303132333435363738394142434445BD
:105690004600286E756C6C20706F696E7465722997
:1056A00000303132333435363738396162636465FE
:0A56B00066003F3F3F0001000000CC
:0400000300000000F9
:00000001FF
